:1028A800EFD3940740037F0122121AEDFED394035D
:1028B80040037F0222EF7041EE700B900001121B63
:1028C80006F452935294121AEDB4010B90000112BF
:1028D8001B064293F45294121AEDFEB4020A9000B9
:1028E80001121B0642934294EEB4030D90000112AC
:1028F8001B06FEF45293EE4294EF64017043121AE1
:10290800EDFE700B900001121B06F452915292EEEC
:10291800B4010B900001121B064291F45292121A54
:10292800EDB4020A900001121B0642914292121A5B
:10293800EDB4030D900001121B06FEF45291EE4215
:1029480092EF64027043121AEDFE700B90000112B0
:102958001B06F452955296EEB4010B900001121B1F
:10296800064295F45296121AEDB4020A900001122A
:102978001B0642954296121AEDB4030D90000112FF
:102988001B06FEF45295EE4296EF64037043121A4A
:10299800EDFE700B900001121B06F452B152B2EE1C
:1029A800B4010B900001121B0642B1F452B2121A84
:1029B800EDB4020A900001121B0642B142B2121A8B
:1029C800EDB4030D900001121B06FEF452B1EE4265
:1029D800B2EF64047043121AEDFE700B90000112FE
:1029E8001B06F452B352B4EEB4010B900001121B53
:1029F8000642B3F452B4121AEDB4020A900001125E
:102A08001B0642B342B4121AEDB4030D9000011232
:102A18001B06FEF452B3EE42B4EF64057043121A7B
:102A2800EDFE700B900001121B06F452C952CAEE5B
:102A3800B4010B900001121B0642C9F452CA121AC3
:102A4800EDB4020A900001121B0642C942CA121ACA
:102A5800EDB4030D900001121B06FEF452C9EE42BC
:102A6800CAEF64067043121AEDFE700B9000011253
:102A78001B06F452CB52CCEEB4010B900001121B92
:102A88000642CBF452CC121AEDB4020A900001129D
:102A98001B0642CB42CC121AEDB4030D9000011272
:102AA8001B06FEF452CBEE42CCEF64077043121AB9
:102AB800EDFF700B900001121B06F452E152E2EF99
:102AC800B4010B900001121B0642E1F452E2121A03
:102AD800EDB4020A900001121B0642E142E2121A0A
:102AE800EDB4030D900001121B06FFF452E1EF4212
:042AF800E27F002257
:0A000E004D435520537461727400D5
:0300B600014A00FC
:103C9D00750903E4F508FB7A0079087F030228A86B
:103B0E00750840750901750D00750CC2750B0175B0
:103B1E000A00750F01E4F510751101F512F513FB8E
:093B2E007A0079087F0102225A95
:103C8C00750801E4F509750A04FB7A007908023B12
:013C9C0037F0
:1038220012399E123B601235D5122FC1123BF4128F
:103832003C15123C9D123B0E123C8C5387EF75FFD8
:1038420041D2AFE54B60097BFF7A00790E123C66EC
:10385200120003054AE54AB40102D290E54AB408CF
:1038620002C290E54AB40A03E4F54A123274120025
:10387200FE121DD81210D61237BC122CB4123354B9
:0538820012313980CB7A
:0C00B900012C00042D00000000011D00BF
:08225A008F148B158A168917F9
:10226200E51464016003022429751E01F51FF5209F
:10227200F521F522F523F524F51874412518F58288
:10228200E43402F583E4F00518E518B420ECE4F533
:102292001874012518F582E43402F583E4F0051878
:1022A200E518B420ECAB15AA16A91790000A121B68
:1022B20006FED3940340037F0222EE700553B7EF6C
:1022C200C2BC90000A121B06B4010553B7EFD2BC80
:1022D20090000A121B06FFB4020543B710C2BCEFFE
:1022E200B4030543B710D2BC121AEDD394C0400315
:1022F2007F0222121AEDFFE598543F4FF598EF64E2
:10230200C06008EF644060030223BE900002121C0A
:10231200D07F007E607D547C00121C0C8F1C8E1BB3
:102322008D1A8C19E4FFFE7D01FCAB1CAA1BA91AB5
:10233200A819C3121CAC40037F0222C3E4951CF50A
:102342001CE4951BF51B7401951AF51AE49519F511
:1023520019AB15AA16A917900001121B06FB6401FE
:10236200702CC28E538EFE5389BF5389CF438E4049
:10237200AF1CAE1BAD1AAC197808121CBD8F8D852F
:102382001C8BC2AB5389BF538FFDD28E8062EB642C
:10239200027026538EEF438E01538EF7438E04AFA5
:1023A2001CAE1BAD1AAC197808121CBD8FD6851C49
:1023B200D753AFFB438E1080377F0222AB15AA168C
:1023C200A917121AEDFF7013900008121B06B40130
:1023D20005438E20801A538EDF8015EFB480119052
:1023E2000008121B06B40105438780800353877FD0
:1023F200AB15AA16A917900009121B06B40104D244
:10240200AC8002C2AC900007121B06B40104D29C3D
:102412008002C29C90000B121B0654C0FFE5A2541E
:102422003F4FF5A27F0022E514640360030225B248
:10243200752503F526F527F528F529F52AF52BF557
:102442001874612518F582E43402F583E4F0051866
:10245200E518B420ECE4F51874212518F582E4346B
:1024620002F583E4F00518E518B420ECAB15AA16C2
:10247200A917121AEDFF64C06008EF6440600302FE
:10248200257490000A121B06FED3940340037F02B8
:1024920022EE700653EEFE53DFFE90000A121B0678
:1024A200B4010653EEFE43DF0190000A121B06FF41
:1024B200B4020643EE0153DFFEEFB4030643EE011E
:1024C20043DF01121AEDB4C00543AC80800353AC64
:1024D2007F900002121CD07F007E607D547C00122F
:1024E2001C0C8F1C8E1B8D1A8C19E4FFFE7D01FCC7
:1024F200AB1CAA1BA91AA819C3121CAC40037F0269
:1025020022C3E4951CF51CE4951BF51B7401951A76
:10251200F51AE49519F519AB15AA16A91790000139
:10252200121B06FBB4031D43AC40AF1CAE1BAD1A1D
:10253200AC197808121CBD8FD4851CD553D1F04339
:10254200D10A8031EB64027026538EEF53ACBF5335
:102552008EF7438E04AF1CAE1BAD1AAC197808126D
:102562001CBD8FD6851CD753AFFB438E1080067FD0
:1025720002227F0222AB15AA16A917900009121B8C
:1025820006B4010543AF08800353AFF7900007126A
:102592001B06B4010543AC10800353ACEF90000B53
:1025A200121B065402FFE5BA54FD4FF5BA7F002212
:0225B2007F02A6
:0125B4002204
:103BAE0074412520F582E43402F583EFF00520E51B
:103BBE0020C394204003E4F520E521700575210112
:033BCE00D2992267
:103C6600121AEDFF600C123BAE740129F9E43AFA20
:033C760080EE22BB
:063BD1008B478A48894978
:103BD700E4FEEEC39D5015AB47AA48A9498E8275EE
:0C3BE7008300121B06FF123BAE0E80E6AE
:013BF30022AF
:030023000234BDE7
:0D34BD00C0E0C083C082C0D075D000C00741
:1034CA00309847C298752C0185463085452F85442A
:1034DA002E85432DE5247032AF99E522C39420400E
:1034EA0003752200BF4404051D8003751D00E51DF8
:1034FA00B40A0375C760AF22052274012FF582E46E
:10350A003402F583E599F0752305309927C299E5C8
:10351A001F6520601C7441251FF582E43402F5837F
:10352A00E0F599051FE51FC394204008751F008028
:04353A0003752100F4
:0B353E00D007D0D0D082D083D0E03284
:1000660074612527F582E43402F583EFF00527E570
:1000760027C394204003E4F527E528700675280178
:0400860043AC022263
:103C7900121AEDFF600C120066740129F9E43AFA90
:033C890080EE22A8
:063B88008B098A0A890B7B
:103B8E00E4FEEEC39D5018AB09050BE50BAA0A70B7
:0F3B9E0002050A14F9121AEDFF1200660E80E3F9
:013BAD0022F5
:03008B0002365CDE
:10365C00C0E0C083C082C0D075D000C007E5AC30DC
:10366C00E034752C0185463085452F85442E8543E5
:10367C002D53ACFEE52B701EE529C3942040037539
:10368C002900AF29052974212FF582E43402F58332
:10369C00E5ADF0752A05E5AC30E12853ACFDE52627
:1036AC006527601C74612526F582E43402F583E0FD
:1036BC00F5AD0526E526C394204008752600800349
:0E36CC00752800D007D0D0D082D083D0E03255
:103B6000750840750903750D00750CC2750B01755C
:103B70000A00750F01751101E4F512751302FB7A45
:083B80000079087F0302225ABC
:1038870064617461206F6B0061736B0070657263B4
:10389700656E74006368616E6765206C696768743C
:1038A70000676C6F62616C206C696768740073777E
:1038B7006974636820737461746500646562756711
:1038C7000076657273696F6E0073686F727420613A
:1038D7006E737765720076657273696F6E5F616E7E
:0538E70073776572001B
:0300C500014B00EC
:10327400E4F508F5099000C8F0E52C640160030248
:103284003353C3E5469530FFE545952FFEE5449558
:103294002EFDE543952DFCE47B08FAF9F8C3121CD6
:1032A400AC4003023353E4F52C852908FFEFC395A2
:1032B40029501B74212FF582E43402F583E0FE7457
:1032C400C92FF582E43400F583EEF00F80DFE4F5D6
:1032D40029FE7F20FD7B017A027921121D76E4FF0D
:1032E4009000CDE0FEEFC39E501274C92FF582E426
:1032F4003400F583E02509F5090F80E4E509F4704D
:103304004EE5086E70499000CCE064017041900075
:10331400CBE0640370399000CAE0540F9000C7F00A
:103324009000CAE020E60280189000C6E0FFA3E007
:10333400B5070EE4A3F09000EF74F0F0900105805F
:0F334400039000C87401F09000C7E09000C6F03D
:013353002257
:1000FE009000C8E070030210D5E54B60097BFF7AD3
:10010E00387987123C669000CFE024E0B4070040B7
:10011E00030210D090013075F003A4C58325F0C5FD
:10012E00837302014502015E020823020A6C020D6E
:10013E00DA0210960210B7E54B60097BFF7A387928
:10014E008F123C669000F67430F09001040210B2EB
:10015E009000EF7431F0E54B60097BFF7A387993AC
:10016E00123C66E4F50874017E00A808088005C3F9
:10017E0033CE33CED8F9FF9000D0E0FDEF5D7003A3
:10018E000204BCE50825E02400F582E43400F58382
:10019E00E4F0A304F0E50825E02418F582E4340029
:1001AE00F583E4F0A3F0C374159508FFE49400FE04
:1001BE0074C92FF58274003EF583E0FFE50825E053
:1001CE002448F582E43400F583E4F0A3EFF0E5086B
:1001DE0025E02448F582E43400F583E0FEA3E0FF39
:1001EE009000ACE0FCA3E0FDC3EF9DEE9C5012E549
:1001FE000825E02448F582E43400F583ECF0A3ED05
:10020E00F0E50825E02448F582E43400F583E0FEAD
:10021E00A3E0FF9000AAE0FCA3E0FDD3EF9DEE9CCF
:10022E004012E50825E02448F582E43400F583EC1D
:10023E00F0A3EDF0E50825E02448F582E43400F55E
:10024E0083E0FEA3E0FF7C047DE2121D49A804A911
:10025E0005AA06AB079000A8E0FEA3E0FFE4FCFDB4
:10026E00121B81E47B64FAF9F8121C0CE47B64FA2D
:10027E00F9F8121C0CA804A905AA06AB07E5082577
:10028E00E024AEF582E43400F583E0FEA3E0FFE463
:10029E00FCFD121B81C374E29FFF74049EFEE508F1
:1002AE0025E02470F582E43401F583EEF0A3EFF03F
:1002BE00E50825E02410F582E43401F583E0FCA383
:1002CE00E0FDE4121A33E50825E025E02440F5822E
:1002DE00E43401F583121D009000D2E075F00AA4FB
:1002EE00FFE50825E02430F582E43400F583E5F0DF
:1002FE00F0A3EFF0E50825E02430F582E43400F5B4
:10030E0083E0FEA3E04E7012E50825E02430F5826E
:10031E00E43400F583E4F0A304F0E50825E02410AE
:10032E00F582E43401F583E0FEA3E0FFE50825E065
:10033E002470F582E43401F583E0FCA3E0FDD39F45
:10034E00EC9E50030203F3E50825E02410F582E449
:10035E003401F583E0FEA3E0FFC3ED9FFDEC9EFCB0
:10036E00E4121A33C004C005C006C007E50825E034
:10037E002430F582E43400F583E0FCA3E0FDE412C2
:10038E001A33A804A905AA06AB07D007D006D005D4
:10039E00D004121924E50825E025E024D0F582E4E6
:1003AE003401F583121D00E50825E025E024D0F583
:1003BE0082E43401F583E0FCA3E0FDA3E0FEA3E0BC
:1003CE00FFE4FBFA7980783F1219C160184016E5F8
:1003DE000825E025E024D0F582E43401F583121DD2
:1003EE000C3F800000E50825E02410F582E434017E
:1003FE00F583E0FEA3E0FFE50825E02470F582E436
:10040E003401F583E0FCA3E0FDC39FEC9E400302A4
:10041E0004BCE50825E02410F582E43401F583E000
:10042E00FEA3E0C39DFDEE9CFCE4121A33C004C093
:10043E0005C006C007E50825E02430F582E4340047
:10044E00F583E0FCA3E0FDE4121A33A804A905AA83
:10045E0006AB07D007D006D005D004121924E50844
:10046E0025E025E024D0F582E43401F583121D0049
:10047E00E50825E025E024D0F582E43401F583E09B
:10048E00FCA3E0FDA3E0FEA3E0FFE4FBFA79807895
:10049E003F1219C160184016E50825E025E024D06A
:1004AE00F582E43401F583121D0C3F80000005082F
:1004BE00E50864086003020174E4F50874017E0027
:1004CE00A808088005C333CE33CED8F9FF9000D1EB
:1004DE00E0FDEF5D7003020812E50825E02410F53B
:1004EE0082E43400F583E4F0A304F0E50825E0246B
:1004FE0028F582E43400F583E4F0A3F0C3740D957F
:10050E0008FFE49400FE74C92FF58274003EF58353
:10051E00E0FFE50825E02458F582E43400F583E495
:10052E00F0A3EFF0E50825E02458F582E43400F559
:10053E0083E0FEA3E0FF9000ACE0FCA3E0FDC3EF80
:10054E009DEE9C5012E50825E02458F582E4340017
:10055E00F583ECF0A3EDF0E50825E02458F582E4F0
:10056E003400F583E0FEA3E0FF9000AAE0FCA3E0D8
:10057E00FDD3EF9DEE9C4012E50825E02458F58250
:10058E00E43400F583ECF0A3EDF0E50825E0245803
:10059E00F582E43400F583E0FEA3E0FF7C047DE207
:1005AE00121D49A804A905AA06AB079000A8E0FEF3
:1005BE00A3E0FFE4FCFD121B81E47B64FAF9F81260
:1005CE001C0CE47B64FAF9F8121C0CA804A905AA09
:1005DE0006AB07E50825E024BEF582E43400F5837A
:1005EE00E0FEA3E0FFE4FCFD121B81C374E29FFF5B
:1005FE0074049EFEE50825E02480F582E43401F5BE
:10060E0083EEF0A3EFF0E50825E02410F582E43444
:10061E0001F583E0FCA3E0FDE4121A33E50825E0C2
:10062E0025E02440F582E43401F583121D0090008C
:10063E00D2E075F00AA4FFE50825E02440F582E437
:10064E003400F583E5F0F0A3EFF0E50825E0244053
:10065E00F582E43400F583E0FEA3E04E7012E50867
:10066E0025E02440F582E43400F583E4F0A304F0A1
:10067E00E50825E02420F582E43401F583E0FEA3AD
:10068E00E0FFE50825E02480F582E43401F583E0FF
:10069E00FCA3E0FDD39FEC9E5003020749E508251D
:1006AE00E02420F582E43401F583E0FEA3E0FFC3ED
:1006BE00ED9FFDEC9EFCE4121A33C004C005C0068B
:1006CE00C007E50825E02440F582E43400F583E018
:1006DE00FCA3E0FDE4121A33A804A905AA06AB0791
:1006EE00D007D006D005D004121924E50825E02540
:1006FE00E024F0F582E43401F583121D00E50825AF
:10070E00E025E024F0F582E43401F583E0FCA3E07B
:10071E00FDA3E0FEA3E0FFE4FBFA7980783F121917
:10072E00C160184016E50825E025E024F0F582E4C6
:10073E003401F583121D0C3F800000E50825E024EE
:10074E0020F582E43401F583E0FEA3E0FFE5082501
:10075E00E02480F582E43401F583E0FCA3E0FDC3E0
:10076E009FEC9E4003020812E50825E02420F58246
:10077E00E43401F583E0FEA3E0C39DFDEE9CFCE4B2
:10078E00121A33C004C005C006C007E50825E024D0
:10079E0040F582E43400F583E0FCA3E0FDE4121A98
:1007AE0033A804A905AA06AB07D007D006D005D0FA
:1007BE0004121924E50825E025E024F0F582E4343E
:1007CE0001F583121D00E50825E025E024F0F582F1
:1007DE00E43401F583E0FCA3E0FDA3E0FEA3E0FF1B
:1007EE00E4FBFA7980783F1219C160184016E508CB
:1007FE0025E025E024F0F582E43401F583121D0C8A
:10080E003F8000000508E508640460030204CA90F6
:10081E0001050210B29000EF7432F0E54B60097BD7
:10082E00FF7A38799B123C66E4F50874017E00A8C5
:10083E0008088005C333CE33CED8F9FF9000D0E040
:10084E00FDEF5D7003020943E50825E02400F58203
:10085E00E43400F583E4F0A3F0E50825E02418F570
:10086E0082E43400F583E4F0A304F09000D2E0FFBC
:10087E00E50825E02460F582E43400F583E4F0A376
:10088E00EFF09000D4E0FFE50825E02490F582E437
:10089E003400F583E4F0A3EFF0E50825E02460F5DD
:1008AE0082E43400F583E0FEA3E04E6003020943C8
:1008BE009000D3E0FF7011E50825E02478F582E47E
:1008CE003400F583E4F0A3F0EFB40112E50825E05F
:1008DE002478F582E43400F583E4F0A304F090006C
:1008EE00D3E06402704FE50825E02478F582E43405
:1008FE0000F583E0FEA3E064014E7013E50825E0E9
:10090E002478F582E43400F583E4F0A3F08026E544
:10091E000825E02478F582E43400F583E0FEA3E0B8
:10092E004E7012E50825E02478F582E43400F58354
:10093E00E4F0A304F00508E5086408600302083932
:10094E00E4F50874017E00A808088005C333CE3391
:10095E00CED8F9FF9000D1E0FDEF5D7003020A5B87
:10096E00E50825E02410F582E43400F583E4F0A3D5
:10097E00F0E50825E02428F582E43400F583E4F060
:10098E00A304F09000D2E0FFE50825E02470F58284
:10099E00E43400F583E4F0A3EFF09000D4E0FFE53B
:1009AE000825E024A0F582E43400F583E4F0A3EFFB
:1009BE00F0E50825E02470F582E43400F583E0FECE
:1009CE00A3E04E6003020A5B9000D3E0FF7011E5D6
:1009DE000825E02488F582E43400F583E4F0A3F0E2
:1009EE00EFB40112E50825E02488F582E43400F521
:1009FE0083E4F0A304F09000D3E06402704FE508A6
:100A0E0025E02488F582E43400F583E0FEA3E0645B
:100A1E00014E7013E50825E02488F582E43400F5D4
:100A2E0083E4F0A3F08026E50825E02488F582E42F
:100A3E003400F583E0FEA3E04E7012E50825E024B5
:100A4E0088F582E43400F583E4F0A304F00508E5AC
:100A5E0008640460030209519001050210B290006F
:100A6E00EF7433F0E54B60097BFF7A3879A8123CBE
:100A7E00669000D0E030E54A9000D3E0FF9000ACE5
:100A8E00E4F0A3EFF0E4F508E50825E02488F5820C
:100A9E00E43401F583E0FEA3E0FF9000ACE0FCA39C
:100AAE00E0FDC3EF9DEE9C5012E50825E02488F58D
:100ABE0082E43401F583ECF0A3EDF00508E508B40B
:100ACE000CC69000D0E030E64A9000D2E0FF9000D5
:100ADE00AAE4F0A3EFF0E4F508E50825E02488F594
:100AEE0082E43401F583E0FEA3E0FF9000AAE0FC6F
:100AFE00A3E0FDD3EF9DEE9C4012E50825E024888F
:100B0E00F582E43401F583ECF0A3EDF00508E50879
:100B1E00B40CC69000D0E020E703020DD4A3E0FF92
:100B2E009000A8E4F0A3EFF0E4F508E50825E02432
:100B3E0000F582E43400F583E4F0A304F0E5082523
:100B4E00E02418F582E43400F583E4F0A3F0E50820
:100B5E0025E02448F582E43400F583E0FEA3E0FFAF
:100B6E007C047DE2121D49A804A905AA06AB0790D4
:100B7E0000A8E0FEA3E0FFE4FCFD121B81E47B6411
:100B8E00FAF9F8121C0CE47B64FAF9F8121C0CA8A2
:100B9E0004A905AA06AB07E50825E024AEF582E414
:100BAE003400F583E0FEA3E0FFE4FCFD121B81C3DD
:100BBE0074E29FFF74049EFEE50825E02470F58222
:100BCE00E43401F583EEF0A3EFF0E50825E0241000
:100BDE00F582E43401F583E0FCA3E0FDE4121A3360
:100BEE00E50825E025E02440F582E43401F5831282
:100BFE001D00E50825E02470F582E43401F583E05C
:100C0E00FEA3E0FFE4FCFD7BE27A04F9F8C3121CBC
:100C1E00AC5014E50825E02470F582E43401F58328
:100C2E007404F0A374E2F0E50825E02410F582E4E4
:100C3E003401F583E0FEA3E0FFE50825E02470F51E
:100C4E0082E43401F583E0FCA3E0FDD39FEC9E50DB
:100C5E0003020D00E50825E02410F582E43401F5C9
:100C6E0083E0FEA3E0FFC3ED9FFDEC9EFCE4121AB1
:100C7E0033C004C005C006C007E50825E02430F5E2
:100C8E0082E43400F583E0FCA3E0FDE4121A33A8FD
:100C9E0004A905AA06AB07D007D006D005D00412CA
:100CAE001924E50825E025E024D0F582E43401F589
:100CBE0083121D00E50825E025E024D0F582E434FA
:100CCE0001F583E0FCA3E0FDA3E0FEA3E0FFE4FB5F
:100CDE00FA7980783F1219C160184016E50825E0B0
:100CEE0025E024D0F582E43401F583121D0C3F80FB
:100CFE000000E50825E02410F582E43401F583E0D8
:100D0E00FEA3E0FFE50825E02470F582E43401F54A
:100D1E0083E0FCA3E0FDC39FEC9E4003020DC9E5FA
:100D2E000825E02410F582E43401F583E0FEA3E00B
:100D3E00C39DFDEE9CFCE4121A33C004C005C00630
:100D4E00C007E50825E02430F582E43400F583E0A1
:100D5E00FCA3E0FDE4121A33A804A905AA06AB070A
:100D6E00D007D006D005D004121924E50825E025B9
:100D7E00E024D0F582E43401F583121D00E5082548
:100D8E00E025E024D0F582E43401F583E0FCA3E015
:100D9E00FDA3E0FEA3E0FFE4FBFA7980783F121991
:100DAE00C160184016E50825E025E024D0F582E460
:100DBE003401F583121D0C3F8000000508E5086420
:100DCE000C6003020B399001050210B29000EF7413
:100DDE0034F0E54B60097BFF7A3879B5123C66E456
:100DEE00F50874017E00A808088005C333CE33CE03
:100DFE00D8F9FF9000D0E0FDEF5D7003020F2D7467
:100E0E00D22508F582E43400F583E0B40117E50835
:100E1E0025E024AEF582E43400F583E4F0A304F07B
:100E2E00AF081238EC74D22508F582E43400F5834D
:100E3E00E0704BAF08123C52E50825E02400F58225
:100E4E00E43400F583E4F0A3F0E50825E02418F57A
:100E5E0082E43400F583E4F0A3F0E50825E0246095
:100E6E00F582E43400F583E4F0A37402F0E508257E
:100E7E00E024AEF582E43400F583E4F0A3F074D2FE
:100E8E002508F582E43400F583E064026003020F66
:100E9E002DE50825E024AEF582E43400F583E0FE6E
:100EAE00A3E04E7019E50825E024AEF582E4340087
:100EBE00F583E4F0A304F0AF081238EC8061E50886
:100ECE0025E024AEF582E43400F583E0FEA3E06471
:100EDE00014E704BAF08123C52E50825E02400F598
:100EEE0082E43400F583E4F0A3F0E50825E024184D
:100EFE00F582E43400F583E4F0A3F0E50825E02460
:100F0E0060F582E43400F583E4F0A37402F0E508A2
:100F1E0025E024AEF582E43400F583E4F0A3F00579
:100F2E0008E508C394085003020DF0E4F5087401B7
:100F3E007E00A808088005C333CE33CED8F9FF90C3
:100F4E0000D1E0FDEF5D700302108574DA2508F51F
:100F5E0082E43400F583E0B4011AE50825E024BEEE
:100F6E00F582E43400F583E4F0A304F0E5082408E8
:100F7E00FF1238EC74DA2508F582E43400F583E0CC
:100F8E00704EE5082408FF123C52E50825E02410B7
:100F9E00F582E43400F583E4F0A3F0E50825E024BF
:100FAE0028F582E43400F583E4F0A3F0E50825E0AB
:100FBE002470F582E43400F583E4F0A37402F0E5C6
:100FCE000825E024BEF582E43400F583E4F0A3F0B6
:100FDE0074DA2508F582E43400F583E064026003D8
:100FEE00021085E50825E024BEF582E43400F58381
:100FFE00E0FEA3E04E701CE50825E024BEF582E479
:10100E003400F583E4F0A304F0E5082408FF123859
:10101E00EC8064E50825E024BEF582E43400F58317
:10102E00E0FEA3E064014E704EE5082408FF123C7A
:10103E0052E50825E02410F582E43400F583E4F04F
:10104E00A3F0E50825E02428F582E43400F583E4D6
:10105E00F0A3F0E50825E02470F582E43400F58372
:10106E00E4F0A37402F0E50825E024BEF582E43432
:10107E0000F583E4F0A3F00508E508C394045003DB
:10108E00020F3C900105801C9000EF7435F0E54B8B
:10109E0060097BFF7A3879C2123C669000D0E0F589
:1010AE004B9001057401F0801990010D7436F0908B
:1010BE0001067401F0E54B60097BFF7A3879C8129E
:0710CE003C66E49000C8F04D
:0110D50022F8
:102CB400E4FFF508900104E07003022D6A9000F02F
:102CC4007401F09000C7E09000F1F0A37403F09059
:102CD40000C9E09000F3F0A37414F09000A8A3E0FE
:102CE4009000F7F0EFFDC3740B9DFDE49400FC909D
:102CF400018875F002ED121D3DEC25E02583F58376
:102D0400A3E0FE74F82FF582E43400F583EEF0EFCF
:102D140025E024AEF582E43400F583E0FCA3E0640E
:102D2400014C700E74F82FF582E43400F583E0440E
:102D340080F00FBF0CAE7B017A0079F07D14123A5B
:102D4400E48F089000F5E508F07B017A0079F07DC6
:102D540014123B88E4900104F0FE7F20FD7B017A8D
:102D64000079C9121D76900105E0605A9000E9745B
:102D740001F09000C7E09000EAF0A37403F0900023
:102D8400C9E09000ECF0A37407F07B017A0079E9C4
:102D9400FD123AE48F089000EEE508F07B017A001A
:102DA40079E97D07123B88E54B60097BFF7A387926
:102DB400D0123C66E4900105F0FE7F20FD7B017A91
:102DC4000079C9121D76900106E06062A37401F0D7
:102DD4009000C7E0900108F0A37403F09000C9E0EC
:102DE40090010AF0A37409F090010E7413F0E4A3A7
:102DF400F07B017A0179077D09123AE48F0890018A
:102E04000CE508F07B017A0179077D09123B88E51E
:102E14004B60097BFF7A3879DD123C66E490010649
:102E2400F0FE7F20FD7B017A0079C9121D767E00B9
:0D2E34007F277D007B017A0079E9021D7681
:063AE4008B098A0A890B20
:103AEA00E4FFFEEEC39D5018EE64056010AB09AA10
:103AFA000AA90B8E82758300121B062FFF0E80E324
:033B0A00EFF4FFD6
:013B0D002295
:0C00C800043B00000000043F00000000AA
:10399E00750903E4F508FB7A0079087F051228A85B
:1039AE007509FF7508037B007A007908E4FF122879
:1039BE00A875090F7508037B007A0079087F02123B
:1039CE0028A87509017508037B007A0079087F0124
:0339DE000228A814
:102FC100750801750D04750EE2E4F50BF50C750A33
:102FD10001FB7A007908FF122AFC7B007A0079084C
:102FE1007F02122AFC7DE37C04E4FF12394A7DE36F
:102FF1007C047F0112394A7DE37C047F0212394A45
:103001007DE37C047F0312394A7DE37C047F041253
:10301100394A7DE37C047F0512394A7DE37C047FD4
:103021000612394A7DE37C047F0712394A7DE37C2D
:10303100047F1012394A7DE37C047F1112394A7DE5
:10304100E37C047F1212394A7DE37C047F13123939
:103051004A7E007FF17D007B017A017910121D7695
:10306100E4FFEF25E02410F582E43401F5837404D4
:10307100F0A374E3F00FBF0CE9E4F512F513F514B6
:103081007B017D01FF1236DAE4F512F513F5147BAD
:10309100017D017F011236DAE4F512F513F5147B97
:1030A100017D017F021236DAE4F512F513F5147B86
:1030B100017D017F031236DAE4F512F513F5147B75
:1030C100017D017F041236DAE4F512F513F5147B64
:1030D100017D017F051236DAE4F512F513F5147B53
:1030E100017D017F061236DAE4F512F513F5147B42
:1030F100017D017F071236DAE4F512F513F5147B31
:10310100017D017F101236DAE4F512F513F5147B17
:10311100017D017F111236DAE4F512F513F5147B06
:10312100017D017F121236DAE4F512F513F5147BF5
:08313100017D017F130236DA73
:101DD800E4F508F509C3E546953EFFE545953DFE62
:101DE800E544953CFDE543953BFCE47B0AFAF9F8AC
:101DF800D3121CAC400302225985463E85453D85D9
:101E0800443C85433BE4F508F509E50925E0FFE591
:101E18000833FE74002FF58274003EF583E0FEA3BC
:101E2800E04E7003022248E50925E0FFE50833FE8D
:101E380074102FF58274013EF583E0FCA3E0FD7475
:101E4800702FF58274013EF583E0FEA3E0D39DEE8A
:101E58009C5003021FCEE509AE087802C333CE3387
:101E6800CED8F92440F58274013EF583C083C08240
:101E7800E0FCA3E0FDA3E0FEA3E0FFC004C005C0B2
:101E880006C007E509AE087802C333CE33CED8F9C9
:101E980024D0F58274013EF583E0F8A3E0F9A3E0CD
:101EA800FAA3E0FBD007D006D005D004121830D032
:101EB80082D083121D00E509AE087802C333CE3301
:101EC800CED8F92440F58274013EF583E0FCA3E006
:101ED800FDA3E0FEA3E0FF121A6CAD07AC06E5090E
:101EE80025E0FFE50833FE74102FF58274013EF5F6
:101EF80083ECF0A3EDF09000A8E07002A3E070106E
:101F080074882FF58274013EF583E4F0A3F08071A4
:101F1800E50925E0FFE50833FE74102FF58274010A
:101F28003EF583E0FEA3E0FBC374E29BFF74049ECE
:101F3800FEE49400FDE49400FCE47B107A27F9F8B1
:101F4800121B81E47BE27A04F9F8121C0CC006C06B
:101F5800079000A8E0FEA3E0FBAA06E4F9F8D00782
:101F6800D006121C0CAD07AC06E50925E0FFE50814
:101F780033FE74882FF58274013EF583ECF0A3EDEF
:101F8800F0E50925E0FFE50833FE74102FF58274AB
:101F9800013EF583E0FCA3E0FD74702FF582740127
:101FA8003EF583E0FAA3E0FBC39DEA9C5018E509DF
:101FB80025E0FFE50833FE74102FF58274013EF525
:101FC80083EAF0A3EBF0E50925E0FFE50833FE74AA
:101FD800102FF58274013EF583E0FCA3E0FD7470D8
:101FE8002FF58274013EF583E0FEA3E0C39DEE9CCD
:101FF80040030221E6E509AE087802C333CE33CEAA
:10200800D8F92440F58274013EF583C083C082E08C
:10201800FCA3E0FDA3E0FEA3E0FFC004C005C006EA
:10202800C007E509AE087802C333CE33CED8F92409
:10203800D0F58274013EF583E0F8A3E0F9A3E0FA55
:10204800A3E0FBD007D006D005D00412182CD0820C
:10205800D083121D00E509AE087802C333CE33CE13
:10206800D8F92440F58274013EF583E0FCA3E0FD35
:10207800A3E0FEA3E0FF121A6CAD07AC06E5092544
:10208800E0FFE50833FE74102FF58274013EF583F6
:10209800ECF0A3EDF09000A8E07002A3E0701074DB
:1020A800882FF58274013EF583E4F0A3F08071E592
:1020B8000925E0FFE50833FE74102FF58274013E10
:1020C800F583E0FEA3E0FBC374E29BFF74049EFE6D
:1020D800E49400FDE49400FCE47B107A27F9F812FC
:1020E8001B81E47BE27A04F9F8121C0CC006C007D5
:1020F8009000A8E0FEA3E0FBAA06E4F9F8D007D018
:1021080006121C0CAD07AC06E50925E0FFE508330F
:10211800FE74882FF58274013EF583ECF0A3EDF090
:10212800E50925E0FFE50833FE74702FF582740198
:102138003EF583E0FCA3E0FDE4121A33C004C005B9
:10214800C006C007E509AE087802C333CE33CED83F
:10215800F924D0F58274013EF583E0F8A3E0F9A3F1
:10216800E0FAA3E0FBD007D006D005D0041218305F
:10217800C004C005C006C007E50925E0FFE508332F
:10218800FE74102FF58274013EF583E0FCA3E0FD98
:10219800E4121A33A804A905AA06AB07D007D0068B
:1021A800D005D0041219C15035E50925E0FFE5082E
:1021B80033FE74102FF58274013EF583E4F0A3F02A
:1021C80074702FF58274013EF583E0FCA3E0FD7482
:1021D800102FF58274013EF583ECF0A3EDF0E509CC
:1021E80025E0FFE50833FE74102FF58274013EF5F3
:1021F80083E0FCA3E0FD74702FF58274013EF58343
:10220800E0FEA3E0B50539EEB50435E50925E0FFA4
:10221800E50833FE74482FF58274003EF583E0FC30
:10222800A3E0FD74882FF58274013EF583ECF0A3DA
:10223800EDF074002FF58274003EF583E4F0A3F00E
:102248000509E50970020508640C45086003021ECB
:012258001273
:012259002262
:1010D600E4F508F509C3E5469542FFE5459541FE69
:1010E600E5449540FDE543953FFCE47B0AFAF9F8B3
:1010F600D3121CAC4003021828854642854541851B
:10110600444085433FE4F508F509E50925E0FFE598
:101116000833FE74182FF58274003EF583E0FCA3B5
:10112600E04C700302181774602FF58274003EF5C8
:1011360083E0FEA3E0FFEE6003021817EF147003CE
:1011460002145414700302180024026003021817D4
:10115600E50925E0FFE50833FE74782FF582740073
:101166003EF583E0FEA3E04E600302131C9000AC44
:10117600E0FEA3E0FF7C047DE2121D49A804A90558
:10118600AA06AB079000A8E0FEA3E0FFE4FCFD1270
:101196001B81E47B64FAF9F8121C0CE47B64FAF90F
:1011A600F8121C0CA804A905AA06AB07E50925E058
:1011B600FFE50833FE74AE2FF58274003EF583E03A
:1011C600FEA3E0FFE4FCFD121B81C374E29FFD74E5
:1011D600049EFCE50925E0FFE50833FE74702FF553
:1011E6008274013EF583ECF0A3EDF074902FF58246
:1011F60074003EF583E0FCA3E0FD74102FF58274C5
:10120600013EF583EC8DF0121B339000A8E07002CE
:10121600A3E07019E50925E0FFE50833FE74882F81
:10122600F58274013EF583E4F0A3F08071E50925AB
:10123600E0FFE50833FE74102FF58274013EF58356
:10124600E0FEA3E0FBC374E29BFF74049EFEE494FD
:1012560000FDE49400FCE47B107A27F9F8121B8168
:10126600E47BE27A04F9F8121C0CC006C007900071
:10127600A8E0FEA3E0FBAA06E4F9F8D007D0061220
:101286001C0CAD07AC06E50925E0FFE50833FE7446
:10129600882FF58274013EF583ECF0A3EDF0E509A5
:1012A60025E0FFE50833FE74702FF58274013EF5E4
:1012B60083E0FCA3E0FD74102FF58274013EF583F4
:1012C600E0FEA3E0C39DEE9C404CE50925E0FFE56A
:1012D6000833FE74182FF58274003EF583E4F0A3FC
:1012E600F074702FF58274013EF583E0FCA3E0FDF7
:1012F60074102FF58274013EF583ECF0A3EDF090A7
:1013060000ACE0FCA3E0FD74882FF58274013EF585
:1013160083ECF0A3EDF0E50925E0FFE50833FE7464
:10132600782FF58274003EF583E0FEA3E064014E5B
:1013360060030218179000AAE0FEA3E0FF7C047D7C
:10134600E2121D49A804A905AA06AB079000A8E069
:10135600FEA3E0FFE4FCFD121B81E47B64FAF9F8CE
:10136600121C0CE47B64FAF9F8121C0CA804A905FB
:10137600AA06AB07E50925E0FFE50833FE74AE2FA4
:10138600F58274003EF583E0FEA3E0FFE4FCFD1267
:101396001B81C374E29FFD74049EFCE50925E0FFF2
:1013A600E50833FE74702FF58274013EF583ECF088
:1013B600A3EDF074902FF58274003EF583E0FCA354
:1013C600E0FD74702FF58274013EF583E0FEA3E024
:1013D6002DFDEE3CFCE50925E0FFE50833FE741023
:1013E6002FF58274013EF583E0FEA3E0D39DEE9CCB
:1013F6005013E50925E0FFE50833FE74182FF58242
:101406007400021707E50925E0FFE50833FE7410AE
:101416002FF58274013EF583C083C082E0FCA3E011
:10142600FD74902FF58274003EF583E0FEA3E0FF85
:10143600C3ED9FFFEC9ED082D083F0A3EFF0900027
:10144600A8E07002A3E0700302177A02178DE5097F
:1014560025E0FFE50833FE74782FF58274003EF52B
:1014660083E0FEA3E04E600302161B9000ACE0FE94
:10147600A3E0FF7C047DE2121D49A804A905AA0683
:10148600AB079000A8E0FEA3E0FFE4FCFD121B8181
:10149600E47B64FAF9F8121C0CE47B64FAF9F8129E
:1014A6001C0CA804A905AA06AB07E50925E0FFE57B
:1014B6000833FE74AE2FF58274003EF583E0FEA37A
:1014C600E0FFE4FCFD121B81C374E29FFD74049EE1
:1014D600FCE50925E0FFE50833FE74702FF58274FC
:1014E600013EF583ECF0A3EDF074902FF5827400C5
:1014F6003EF583E0FCA3E0FD74102FF58274013EF7
:10150600F583EC8DF0121B339000A8E07002A3E087
:101516007019E50925E0FFE50833FE74882FF5828A
:1015260074013EF583E4F0A3F08071E50925E0FF40
:10153600E50833FE74102FF58274013EF583E0FE54
:10154600A3E0FBC374E29BFF74049EFEE49400FDDB
:10155600E49400FCE47B107A27F9F8121B81E47B03
:10156600E27A04F9F8121C0CC006C0079000A8E045
:10157600FEA3E0FBAA06E4F9F8D007D006121C0C7D
:10158600AD07AC06E50925E0FFE50833FE74882FB4
:10159600F58274013EF583ECF0A3EDF0E50925E054
:1015A600FFE50833FE74702FF58274013EF583E083
:1015B600FCA3E0FD74102FF58274013EF583E0FE76
:1015C600A3E0C39DEE9C404DE50925E0FFE5083309
:1015D600FE74782FF58274003EF583E4F0A304F0E0
:1015E60074702FF58274013EF583E0FCA3E0FD7470
:1015F600102FF58274013EF583ECF0A3EDF0900018
:10160600ACE0FCA3E0FD74882FF58274013EF583FF
:10161600ECF0A3EDF0E50925E0FFE50833FE74786C
:101626002FF58274003EF583E0FEA3E064014E6070
:10163600030218179000AAE0FEA3E0FF7C047DE2F7
:10164600121D49A804A905AA06AB079000A8E0FE4A
:10165600A3E0FFE4FCFD121B81E47B64FAF9F812B7
:101666001C0CE47B64FAF9F8121C0CA804A905AA60
:1016760006AB07E50925E0FFE50833FE74AE2FF556
:101686008274003EF583E0FEA3E0FFE4FCFD121B3E
:1016960081C374E29FFD74049EFCE50925E0FFE525
:1016A6000833FE74702FF58274013EF583ECF0A3C7
:1016B600EDF074902FF58274003EF583E0FCA3E014
:1016C600FD74702FF58274013EF583E0FEA3E02DD4
:1016D600FDEE3CFCE50925E0FFE50833FE74102F1E
:1016E600F58274013EF583E0FEA3E0D39DEE9C50A7
:1016F60040E50925E0FFE50833FE74782FF582748E
:10170600003EF583E4F0A3F074702FF58274013E79
:10171600F583E0FCA3E0FD74102FF58274013EF51D
:1017260083ECF0A3EDF09000AAE0FCA3E0FD021725
:10173600EFE50925E0FFE50833FE74102FF5827406
:10174600013EF583C083C082E0FCA3E0FD74902FC8
:10175600F58274003EF583E0FEA3E0FFC3ED9FFF34
:10176600EC9ED082D083F0A3EFF09000A8E0700248
:10177600A3E07013E50925E0FFE50833FE74882F22
:10178600F5827401021810E50925E0FFE50833FE2D
:1017960074102FF58274013EF583E0FEA3E0FBC3CF
:1017A60074E29BFF74049EFEE49400FDE49400FC46
:1017B600E47B107A27F9F8121B81E47BE27A04F9BC
:1017C600F8121C0CC006C0079000A8E0FEA3E0FBC0
:1017D600AA06E4F9F8D007D006121C0CAD07AC0631
:1017E600E50925E0FFE50833FE74882FF5827401CC
:1017F6003EF583ECF0A3EDF08017E50925E0FFE563
:101806000833FE74182FF58274003EF583E4F0A3C6
:10181600F00509E50970020508640C450860030235
:0218260011109F
:01182800229D
:103C5200EF25E02410F582E43401F583744EF0A3DD
:043C62007421F022B7
:1038EC008F09EF25E02488F582E43401F583E0FEAE
:1038FC00A3E0FF7C047DE2121D49A804A905AA06D9
:10390C00AB079000A8E0FEA3E0FFE4FCFD121B81D6
:10391C00E47B64FAF9F8121C0CE47B64FAF9F812F3
:10392C001C0CC374E29FFF74049EFEE50925E02481
:0E393C0010F582E43401F583EEF0A3EFF022E3
:103423008C0A8D0BEFB40C0040030234BC9034378C
:10343300F828287302345B02346302346B0234735A
:1034430002347B02348302348B02349302349B02B2
:1034530034A30234AB0234B3AD0BAC0A7F078056FE
:10346300AD0BAC0A7F06804EAD0BAC0A7F058046E0
:10347300AD0BAC0A7F04803EAD0BAC0A7F038036F4
:10348300AD0BAC0A7F02802EAD0BAC0A7F01802608
:10349300AD0BAC0AE4FF801EAD0BAC0A7F138016A4
:1034A300AD0BAC0A7F12800EAD0BAC0A7F11800608
:0A34B300AD0BAC0A7F1012394A225B
:1037BC00E4F508F509E50925E0FFE50833FE74108A
:1037CC002FF58274013EF583E0FEA3E0FFE4FCFDDF
:1037DC007B207A4EF9F8C3121CACAF097005123C71
:1037EC0052801FC007E50925E0FFE50833FE741081
:1037FC002FF58274013EF583E0FCA3E0FDD00712A7
:10380C0034230509E50970020508C3940CE5086426
:05381C0080948040A033
:013821002284
:1035D5007E007F237D007B017A0079C6121D767EF1
:1035E500007FC67D007B017A007900121D767E0082
:1035F5007F277D007B017A0079E9121D769000C650
:1036050074FFF0E49000ACF0A3F09000AAF0A3746E
:1036150064F09000A8E4F0A37464F0E4FFEF25E003
:103625002490F582E43400F583E4F0A304F0EF255B
:10363500E024AEF582E43400F583E4F0A304F0EF72
:1036450025E02430F582E43400F5837401F0A37499
:063655002CF00FBF0CC7B2
:01365B00224C
:103BF400E4F508750903750A01750B01F50C750DDB
:103C0400F8750ECD750F01FB7A0079087F02022545
:013C1400B5FA
:102E4100FF14FF1CFF24FF2CFF34FF3CFF44FF4C09
:102E5100FF64FF6CFF74FF7CFF84FF8CFF94FF9C79
:102E6100FFB4FFBCFFC4FFCCFFD4FFDCFFE4FFECE9
:102E7100FC14FC1CFC24FC2CFC34FC3CFC44FC4CF1
:102E8100FC64FC6CFC74FC7CFC84FC8CFC94FC9C61
:102E9100FCB4FCBCFCC4FCCCFCD4FCDCFCE4FCECD1
:102EA100FF10FF18FF20FF28FF30FF38FF40FF48C9
:102EB100FF60FF68FF70FF78FF80FF88FF90FF9839
:102EC100FFB0FFB8FFC0FFC8FFD0FFD8FFE0FFE8A9
:102ED100FC10FC18FC20FC28FC30FC38FC40FC48B1
:102EE100FC60FC68FC70FC78FC80FC88FC90FC9821
:102EF100FCB0FCB8FCC0FCC8FCD0FCD8FCE0FCE891
:102F0100FF12FF1AFF22FF2AFF32FF3AFF42FF4A58
:102F1100FF62FF6AFF72FF7AFF82FF8AFF92FF9AC8
:102F2100FFB2FFBAFFC2FFCAFFD2FFDAFFE2FFEA38
:102F3100FC12FC1AFC22FC2AFC32FC3AFC42FC4A40
:102F4100FC62FC6AFC72FC7AFC82FC8AFC92FC9AB0
:102F5100FCB2FCBAFCC2FCCAFCD2FCDAFCE2FCEA20
:102F6100FF15FF1DFF25FF2DFF35FF3DFF45FF4DE0
:102F7100FF65FF6DFF75FF7DFF85FF8DFF95FF9D50
:102F8100FFB5FFBDFFC5FFCDFFD5FFDDFFE5FFEDC0
:102F9100FC15FC1DFC25FC2DFC35FC3DFC45FC4DC8
:102FA100FC65FC6DFC75FC7DFC85FC8DFC95FC9D38
:102FB100FCB5FCBDFCC5FCCDFCD5FCDDFCE5FCEDA8
:1036DA00EFD3942F40037F0222EDD3940140037F5E
:1036EA000222EBD3940140037F0222E512D3940114
:1036FA0040037F0222E513D3940140037F0222E5AF
:10370A0014D3940140037F022243BA80EF25E024B8
:10371A0041F582E4342EF583E493FE740193F58235
:10372A008E83EBC4333354C0FFEDC4333333548038
:10373A004FFFE51225E025E04FFFE51325E04F4551
:07374A0014F053BA7F7F0069
:013751002255
:10394A00EFD3942F40037F0222D3ED94FFEC947FB0
:10395A0040037F022243BA80EF25E024A1F582E4E6
:10396A00342EF583E493FA740193F5828A83EC5436
:10397A007FF0A3EDF0EF25E02401F582E4342FF582
:10398A0083E493FE740193F5828E83E4F0A3F053EB
:03399A00BA7FFFF2
:01399D002207
:02375200A907C5
:10375400E9D3942F40037F0222D3ED94FFEC947FAE
:1037640040037F0222D3EB94FFEA947F40037F025D
:103774002243BA80E925E024A1F582E4342EF583BE
:10378400E493FE740193F5828E83EC547FAF05F0CD
:10379400A3EFF0E925E02401F582E4342FF583E476
:1037A40093FE740193F5828E83EA547FAF03F0A3F2
:0737B400EFF053BA7F7F0024
:0137BB0022EB
:1039E100EFD3942F40037F0222EBD3940140037F56
:1039F1000222EDD3940140037F022243BA80EF25D6
:103A0100E02461F582E4342FF583E493FE7401939D
:0E3A1100F5828E83EB25E04DF053BA7F7F00E7
:013A1F002284
:102AFC00EFD394054003022CB343BA80EF7042121B
:102B0C001AEDB4010543F101800353F1FE9000046A
:102B1C00121B06540FFE90FF02E054F04EF0900092
:102B2C0005121B49FDE5F0547F90FF00F0A3EDF07A
:102B3C00900002121B06B4010543F601800353F604
:102B4C00FEEF64017042121AEDB4010543F10280EC
:102B5C000353F1FD900004121B06540FFE90FF521C
:102B6C00E054F04EF0900005121B49FDE5F0547F47
:102B7C0090FF50F0A3EDF0900002121B06B401057B
:102B8C0043F610800353F6EFEF64027042121AED15
:102B9C00B4010543F104800353F1FB900004121BB4
:102BAC0006540FFE90FFA2E054F04EF09000051278
:102BBC001B49FDE5F0547F90FFA0F0A3EDF09000D1
:102BCC0002121B06B4010543F701800353F7FEEF15
:102BDC0064037042121AEDB4010543F108800353EB
:102BEC00F1F7900004121B06540FFE90FC02E05407
:102BFC00F04EF0900005121B49FDE5F0547F90FC5F
:102C0C0000F0A3EDF0900002121B06B4010543F78F
:102C1C0010800353F7EFEF64047042121AEDB40105
:102C2C000543F110800353F1EF900004121B06547E
:102C3C000FFE90FC52E054F04EF0900005121B4930
:102C4C00FDE5F0547F90FC50F0A3EDF090000212E3
:102C5C001B06B4010543FE01800353FEFEEF640521
:102C6C007042121AEDB4010543F120800353F1DFD9
:102C7C00900004121B06540FFF90FCA2E054F04F7E
:102C8C00F0900005121B49FFE5F0547F90FCA0F07A
:102C9C00A3EFF0900002121B06B4010543FE108056
:082CAC000353FEEF53BA7F222F
:0300B30002002622
:0D002600C0E0C083C082C0D075D000C0070C
:10003300AFBA43BA80E5F630E30353F6F790FF0512
:09004300E06004E4F0B2A78FBAFA
:0B004C00D007D0D0D082D083D0E032AB
:0300E300023A20BE
:0D3A2000C0E0C083C082C0D075D000C007D8
:103A2D00AFBA43BA80E5F630E70353F67F90FF5502
:093A3D00E06004E4F0B2A68FBAC7
:0B3A4600D007D0D0D082D083D0E03277
:0300EB00023A5185
:0D3A5100C0E0C083C082C0D075D000C007A7
:103A5E00AFBA43BA80E5F730E30353F7F790FFA50B
:093A6E00E06004E4F0B2A58FBA97
:0B3A7700D007D0D0D082D083D0E03246
:0300F300023A824C
:0D3A8200C0E0C083C082C0D075D000C00776
:103A8F00AFBA43BA80E5F730E70353F77F90FC05F1
:093A9F00E06004E4F0B2A48FBA67
:0B3AA800D007D0D0D082D083D0E03215
:0300FB00023AB313
:0D3AB300C0E0C083C082C0D075D000C00745
:103AC000AFBA43BA80E5FE30E30353FEF790FC55EE
:093AD000E06004E4F0B2A38FBA37
:0B3AD900D007D0D0D082D083D0E032E4
:0600D400044300000000DF
:03000B00020007E9
:03000700B2EF3223
:03001B00020018C8
:03001800B2EE3213
:03006300023C3428
:103C3400C0E0C0D0E5462401F546E43545F545E449
:0E3C44003544F544E43543F543D0D0D0E032AA
:03009B0002000A56
:01000A0032C3
:0300A30002001E3A
:03001E00B2EB3210
:1025B500AD07EDD3940440037F0122ED60030226AD
:1025C50077C28C900002121B06B40104D2A98002C6
:1025D500C2A9900001121B06FED3940340037F029B
:1025E50022EE700553B7FDC2B9900001121B06B467
:1025F500010553B7FDD2B9900001121B06FFB402C5
:102605000543B702C2B9EFB4030543B702D2B91205
:102615001AEDFEC3940340037F0222E58954CF4E91
:10262500F589900003121B06FFB40103538E7FEF5B
:102635007003438E80EFB4020543890480035389F8
:10264500FB900004121B06B40105438F0180035360
:102655008FFE900005121B49E5F0F58C90000512E0
:102665001B49F58A900007121B06B40102D28C7F24
:102675000022ED64016003022730C28E9000021231
:102685001B06B40104D2AB8002C2AB900001121B41
:1026950006FED3940340037F0222EE700553B7F77D
:1026A500C2BB900001121B06B4010553B7F7D2BB9C
:1026B500900001121B06FFB4020543B708C2BBEF29
:1026C500B4030543B708D2BB121AEDFEC394034009
:1026D500037F0222E58954CF4EF589900003121B32
:1026E50006FFB40103538EBFEF7003438E40EFB472
:1026F500020543894080035389BF900004121B06DD
:10270500B40105438F028003538FFD900005121B12
:1027150049E5F0F58D900005121B49F58B900007F2
:10272500121B06B40102D28E7F0022ED640270787E
:10273500538EEF900002121B06B4010543AF0480CF
:102745000353AFFB900003121B06FED39402400314
:102755007F0222EEB40103538EFB900003121B0689
:102765007003438E04900003121B06B40205438ECA
:10277500088003538EF7900004121B06B40105432D
:102785008F048003538FFB900005121B49E5F0F57C
:10279500D6900005121B49F5D7900007121B06B409
:1027A5000103438E107F0022ED6403707853D1F747
:1027B500900002121B06B4010543AF20800353AFFE
:1027C500DF900003121B06FED3940240037F022212
:1027D500EEB4010353D1FD900003121B06700343B1
:1027E500D102900003121B06B4020543D1048003F5
:1027F50053D1FB900004121B06B4010543D101809F
:102805000353D1FE900005121B49E5F0F5D4900065
:1028150005121B49F5D5900007121B06B4010343A9
:10282500D1087F0022ED6404707653D17F900002B9
:10283500121B06B4010543AF40800353AFBF9000A0
:1028450003121B06FED3940240037F0222EEB4015D
:102855000353D1DF900003121B06700343D1209070
:102865000003121B06B4020543D140800353D1BFB8
:10287500900004121B06B4010543D110800353D107
:10288500EF900005121B49FDACF0ECF5D2AF058FBA
:10289500D3900007121B06B4010343D1807F0022A9
:0328A5007F02228D
:0600DA00043100000000EB
:103C1500750910E4F508FB7A0079087F041228A8D5
:0F3C25007E007F067D007B007A007935021D76D8
:10335400C3E5469534FFE5459533FEE5449532FDD6
:10336400E5439531FCE47B0AFAF9F8C3121CAC403E
:1033740003023422854634854533854432854331FE
:10338400E4FF74362FF8E614603A14607324026084
:103394000302341920C41D743A2FF8E6C394025072
:1033A4000306807174362FF8760174392FF8E4F629
:1033B400743A802C743A2FF8E4F674362FF8E4F655
:1033C4007437801C74392FF806E6C39464501730A0
:1033D400C44374372FF8760174392FF8E4F6743641
:1033E4002FF8E4F6802F74362FF8760274392FF80C
:1033F400E4F674382FF8760374372FF876028015C4
:1034040074382FF8E4F630C40C74362FF8E4F674EC
:0E341400372FF876040FEF6401600302338651
:013422002287
:10313900E53764016003023273F537900200E00459
:10314900F0E014B40D00400302327390316275F05F
:1031590003A4C58325F0C58373023189023199021D
:1031690031A90231B90231C80231D70231E602313F
:10317900F50232040232130232220232310232459E
:103189009001107407F0A374D0F090018802323EC8
:103199009001127407F0A374D0F090018A02323EB4
:1031A9009001147407F0A374D0F090018C02323EA0
:1031B9009001167407F0A374D0F090018E80769078
:1031C90001187407F0A374D0F09001908067900102
:1031D9001A7407F0A374D0F0900192805890011CE2
:1031E9007407F0A374D0F0900194804990011E7483
:1031F90007F0A374D0F0900196803A9001207407EB
:10320900F0A374D0F0900198802B9001227407F0FC
:10321900A374D0F090019A801C9001247407F0A344
:1032290074D0F090019C800D9001267407F0A3746E
:10323900D0F090019EE4F0A3745AF022E4FFEF2548
:10324900E02410F582E43401F5837404F0A374E2F8
:10325900F0EF25E02488F582E43401F583E4F0A356
:0A326900F00FBF0CD9E4900200F052
:013273002238
:103B3700121AEDB4010375C120900002121B06543E
:103B470007FFE5C154F84FF5C1900001121B06703D
:093B57000453C1F72243C1082206
:0400030043C11022C3
:10182900021AD8E86480F8E933E83360110460F0FB
:10183900ED33EC337009E8FCE9FDEAFEEBFF220425
:1018490060DED3EB9FEA9EE99DE8C2E78CF0C2F720
:1018590095F0400CE8CCF8E9CDF9EACEFAEBCFFBEC
:10186900121AA385D0F05804700320D5B3E8047088
:10187900075002B2D5021AE292D5EC0460F7E4CC23
:10188900C0E0C398F8603B94186008400DD0E0FBB5
:10189900021ABAE4FBFAC9FC8028E830E406E4C974
:1018A900FBE4CAFCE830E305E4C9CACBFCE8540709
:1018B9006010F8C3E913F9EA13FAEB13FBEC13FC14
:1018C900D8F130F52FC3E49CFCEF9BFFEE9AFEEDB7
:1018D90099FDD0E0FBEF4E4D4C701222DB03021A4A
:1018E900DFEC2CFCEF33FFEE33FEED33FDED30E79B
:1018F900EB021ABAEF2BFFEE3AFEED39FDD0E0FB11
:1019090050130BBB0003021AE2ED13FDEE13FEEFB9
:0819190013FFEC13FC021ABAE3
:10192100021AE2EC5D046005E859047003021AD85A
:10193100121AA3580460F6EC4860F2EC7004FDFE44
:10194100FF22C860DB2481C85009C3986002500699
:10195100021ADF9850CAF582E9294B4A7005AB8219
:10196100021ACE75F0007C1A7880C3EF9BEE9AEDD7
:1019710099400DC3EF9BFFEE9AFEED99FDE842F011
:10198100DC23ACF0D0E0FFD0E0FED0E0FDAB822064
:10199100E7101BEB60BAEC2CFCEF33FFEE33FEEDEE
:1019A10033FD021ABAE803F830E705C0F075F0001C
:1019B100EF2FFFEE33FEED33FD40B830E7C280AAD2
:1019C10074F8CC6480CCC86480C8F582046043C3D9
:1019D100EB9FF5F0EA9E42F0E99D42F0E89C45F06C
:1019E10060305018E5825FFFE582F42B5582FB5091
:1019F100210ABA001D09B90019088016E5825BFBAE
:101A0100E582F42F5582FF50090EBE00050DBD0081
:101A1100010CC3EB9FF5F0EA9E42F0E99D42F0E82C
:0D1A21009C45F06007CC4820E701B3EC22A3
:101A2E0075F020800E75F010800575F0087D007E33
:101A3E00007F003392D530D503121C9EEC3340103C
:101A4E00EF33FFEE33FEED33FDEC33FCD5F0ED223C
:0E1A5E00E5F0247EA2D513CC92E7CDCEFF2278
:101A6C00EDD2E7CD33EC3392D524814006E4FFFE72
:101A7C00FDFC22FCE4CFCECDCC24E0501174FF80D1
:101A8C00EDC3CC13CCCD13CDCE13CECF13CF04706E
:071A9C00F030D5DE021C9EB4
:101AA300E9D2E7C933E833F892D5EDD2E7CD33EC89
:071AB30033FC5002B2D52202
:101ABA00EC30E7100FBF000C0EBE00080DBD00048D
:101ACA000BEB6014A2D5EB13FCED92E7FD2274FF39
:101ADA00FCFDFEFF22E480F8A2D574FF13FC7D8092
:031AEA00E480EFA6
:030000000235497D
:0C354900787FE4F6D8FD75814B023590C8
:101AED00BB010689828A83E0225002E722BBFE02F7
:091AFD00E32289828A83E493222A
:101B0600BB010CE58229F582E5833AF583E0225094
:101B160006E92582F8E622BBFE06E92582F8E222DE
:0D1B2600E58229F582E5833AF583E49322F8
:101B3300C5F0F8A3E028F0C5F0F8E582158270023D
:061B43001583E038F022DA
:101B4900BB0110E58229F582E5833AF583E0F5F0DA
:101B5900A3E0225009E92582F886F008E622BBFEB7
:101B69000AE92582F8E2F5F008E222E5832AF583FD
:081B7900E993F5F0A3E99322C2
:101B8100E88FF0A4CC8BF0A42CFCE98EF0A42CFC03
:101B91008AF0EDA42CFCEA8EF0A4CDA8F08BF0A481
:101BA1002DCC3825F0FDE98FF0A42CCD35F0FCEBE0
:101BB1008EF0A4FEA9F0EB8FF0A4CFC5F02ECD39A5
:0F1BC100FEE43CFCEAA42DCE35F0FDE43CFC2212
:101BD00075F008758200EF2FFFEE33FECD33CDCCCC
:101BE00033CCC58233C5829BED9AEC99E58298404F
:101BF0000CF582EE9BFEED9AFDEC99FC0FD5F0D62C
:101C0000E4CEFBE4CDFAE4CCF9A88222B800C1B955
:101C10000059BA002DEC8BF084CFCECDFCE5F0CB93
:101C2000F97818EF2FFFEE33FEED33FDEC33FCEBCC
:101C300033FB10D703994004EB99FB0FD8E5E4F987
:101C4000FA227818EF2FFFEE33FEED33FDEC33FC74
:101C5000C933C910D7059BE99A4007EC9BFCE99A68
:101C6000F90FD8E0E4C9FAE4CCFB2275F010EF2FAD
:101C7000FFEE33FEED33FDCC33CCC833C810D707AD
:101C80009BEC9AE899400AED9BFDEC9AFCE899F8E8
:0E1C90000FD5F0DAE4CDFBE4CCFAE4C8F9227B
:0E1C9E00C3E49FFFE49EFEE49DFDE49CFC2257
:101CAC00EB9FF5F0EA9E42F0E99D42F0E89C45F08E
:011CBC002205
:101CBD00E8600FECC313FCED13FDEE13FEEF13FF05
:031CCD00D8F12229
:101CD000BB010DE58229F582E5833AF583021DAF4C
:101CE0005007E92582F8021DA2BBFE07E92582F80C
:101CF000021DBBE58229F582E5833AF583021DC802
:0C1D0000ECF0A3EDF0A3EEF0A3EFF02256
:101D0C00A8828583F0D083D082121D23121D23124A
:101D1C001D23121D23E473E493A3C583C5F0C5836F
:101D2C00C8C582C8F0A3C583C5F0C583C8C582C821
:011D3C002284
:0C1D3D00A42582F582E5F03583F58322B1
:101D4900EC8EF0A4CCC5F0CCCDF8EFA4CEC5F02D27
:101D5900FDE43CFCE8A42EC8C5F03DFDE43CFCEFE5
:0D1D6900A4FFE5F028FEE43DFDE43CFC2273
:101D7600EF4E6012EF60010EEDBB010B89828A8384
:101D8600F0A3DFFCDEFA2289F05007F709DFFCA991
:0C1D9600F022BBFEFCF309DFFCA9F022E8
:10355500023822E493A3F8E493A34003F68001F232
:1035650008DFF48029E493A3F85407240CC8C33377
:10357500C4540F4420C8834004F456800146F6DF46
:10358500E4800B01020408102040809000B6E47E20
:10359500019360BCA3FF543F30E509541FFEE4933B
:1035A500A360010ECF54C025E060A840B8E493A302
:1035B500FAE493A3F8E493A3C8C582C8CAC583CA2D
:1035C500F0A3C8C582C8CAC583CADFE9DEE780BEE5
:0100E000001F
:0D1DA200E6FB08E6F908E6FA08E6CBF822B1
:0C1DAF00E0F8A3E0F9A3E0FAA3E0FB22B7
:0D1DBB00E2FB08E2F908E2FA08E2CBF822A8
:101DC800E493F8740193F9740293FA740393FB2271
:00000001FF
